:020000020000FC
:10000000FFC097C397C397C397C397C3B6C435C4FC
:1000100035C435C41CC418C418C418C48FC312C452
:1000200012C4ACC4A3C4A3C4A3C4A9C4A5C4A3C418
:04003000A7C4A7C4F6
:10020000F89400E811E0009361001093610001E0B0
:1002100005B90EEF04B90FE508B900EA07B900E027
:100220000BB90FEF0AB9B1E0A0E0D5E0C0E000E003
:100230000D93BD17E9F7AC17D9F714E00EEF1EBF09
:100240000DBF00E005BF03E00CBB02E004BD03E00E
:1002500005BD00E006BD0FE307BD00E008BD00E0FE
:1002600003BD00E00093800001E40093810000E002
:100270000093820010E000E010938500009384005A
:1002800010E000E0109389000093880010E000E087
:1002900010938B0000938A0010E000E01093870019
:1002A0000093860000E00093B00007E00093B100E7
:1002B00000E00093B20000E00093B30000E0009380
:1002C000B40000E00093B60000E000937C0007E07B
:1002D00000937A0000E000937B0000E000937E0032
:1002E00000E80093300000E000937F0010E003E09E
:1002F0001093C5000093C40002E20093C00000E028
:100300000093C10006E00093C20003E50CBD00E0CD
:100310000DBD0CE00093B80000E00093B90001E7C8
:100320000894001F0093BA0000E00093BC0000E0B6
:1003300000937B0000E00093690009E319E3009358
:1003400060001093600003E80093640000E00DBBC0
:1003500004E00093680000E000936B0000E000936D
:100360006C0000E000936D0002E000936E0000E27C
:1003700000936F0001E00093700007E005BB07E207
:1003800006BB07E007BBB1E0A0E00AE20D930AE27A
:100390000D930EE20D930AE20D930AE20D930AE229
:1003A0000D930DE40D9308E40D930AE70D930AE213
:1003B0000D930AE20D930AE20D930EE70D930AE204
:1003C0000D930AE20D930AE20D930FE40D9303E5FA
:1003D0000D9303E40D9303E40D9301E40D930CE4FA
:1003E0000D930DE30D930AE20D930AE20D930AE2D9
:1003F0000D9308E20D9300E30D9308E70D930AE2D5
:100400000D930AE20D9309E20D9350E040E075D39D
:100410000A3358F4B1E0A0E850E040E01BE06DD3AF
:100420000D9343951A95D9F718C0B1E0A0E800E004
:100430000D9304E00D9300E00D9300E00D9300E0B8
:100440000D9300E00D9300E00D9300E00D9302E0AA
:100450000D9305E00D9305E00D9390E0D1E0C0E829
:1004600000E0E02E04E0D02E0AEF4ED308E1006257
:100470009CD208E1006299D200E0016096D200E0CF
:10048000026093D202E0046090D204E008608DD252
:100490007894A8950091550100FF08C0009156017D
:1004A00000FD09C00160009356014AC00091560149
:1004B0000E7F009356010091550101FF08C0009185
:1004C000560101FD09C00260009356013FC0009132
:1004D00056010D7F009356010091550102FF08C09F
:1004E0000091560102FD09C004600093560134C01A
:1004F000009156010B7F009356010091550103FFB7
:1005000008C00091560103FD09C008600093560120
:1005100027C000915601077F0093560100915501B5
:1005200004FF08C00091560104FD09C0006100935A
:1005300056011AC0009156010F7E00935601F8C073
:100540000881093011F003950883F2C0088100305A
:1005500011F00A950883ECC0CA3809F0C395E8C0C9
:10056000C03809F0CA95E4C0B1E0A0E850E040E02E
:1005700065EA1BE00D91B3D243951A95D9F760E077
:1005800020E010E000E0B1E0A0E860E057E240E1E8
:100590003D91303029F0040F151F261F3A95D9F7E9
:1005A00060E053E048EE3D91303029F0040F151F14
:1005B000261F3A95D9F760E050E044E63D9130308F
:1005C00029F0040F151F261F3A95D9F760E050E077
:1005D0004AE03D91303029F0040F151F261F3A954F
:1005E000D9F760E03D91030F161F261FB1E0A7E188
:1005F0003DE23D933DE23D933DE23D9338E23D9344
:1006000030E33D9338E73D933DE23D933DE23D933A
:1006100039E23D9370E0622F512F402F33E02EE6F8
:1006200018EE00E0D4D1732E622E512E402EB1E090
:10063000A5E82D911D910D91FED1B02EA02EA39471
:10064000A394B1E0A8E82D911D910D91F4D1C02E95
:100650000FEF0093870000938600A89500E00093B9
:100660006E0000E000937000BEBC00918100006449
:100670000093810091FFFECF9D6F80908600909047
:100680008700192D082D352D242DC5D118F4BA1445
:10069000D0F51EC0B394CB14D9F00B2DE0D120932C
:1006A000170110931801009319010B2DEDD1109330
:1006B0001D0100931E0101E0D02E01E0E02E0AEFA3
:1006C0000093B20001E0009370000AE01DD2C5CF94
:1006D000B1E0A7E10DE20D930DE20D930DE20D9354
:1006E00008E20D9300E30D9308E70D930DE20D93DF
:1006F0000DE20D9309E20D9302E000936E0001E01C
:100700000093700015C0BA940B2DA9D12093170146
:1007100010931801009319010B2DB6D110931D01F0
:1007200000931E0102E000936E0001E00093700050
:10073000B0CE18951895189518951895FFB60F9383
:100740001F9306B110915001089400FD8894111F69
:10075000109350011F3F31F4009155010160009347
:10076000550108C0103031F4009155010E7F0093FF
:10077000550100C006B110915101089401FD889403
:10078000111F109351011F3F31F400915501026078
:100790000093550108C0103031F4009155010D7FD0
:1007A0000093550100C006B110915201089402FD5A
:1007B0008894111F109352011F3F31F4009155018D
:1007C00004600093550108C0103031F400915501C8
:1007D0000B7F0093550100C006B11091530108949E
:1007E00003FD8894111F109353011F3F31F40091B2
:1007F000550108600093550108C0103031F4009194
:100800005501077F0093550100C006B110915401B6
:10081000089404FD8894111F109354011F3F31F474
:100820000091550100610093550108C0103031F46A
:10083000009155010F7E0093550100C01F910F914B
:10084000FFBE189518951895189518951895FFB628
:100850000F931F930091810006FF0AC00F7B009346
:10086000810010E000E0109385000093840001C037
:1008700092601F910F91FFBE189518951895FFB6BD
:100880000F931F93AF93BF93DA9409F069C002E00E
:10089000D02EB1E0A0E810E3E3940C91010FAC1767
:1008A00011F4E0FC00E2A395009300010C91010F0C
:1008B000AC1711F4E0FC00E2A395009301010C9148
:1008C000010FAC1711F4E0FC00E2A39500930301C3
:1008D0000C91010FAC1711F4E0FC00E2A39500931A
:1008E00004010C91010FAC1711F4E0FC00E2A39598
:1008F000009305010C91010FAC1711F4E0FC00E22C
:10090000A395009309010C91010FAC1711F4E0FCC1
:1009100000E2A39500930A010C91010FAC1711F4AA
:10092000E0FC00E2A39500930B010C91010FAC17C2
:1009300011F4E0FC00E2A39500930D010C91010F6E
:10094000AC1711F4E0FC00E2A39500930E010C91AA
:10095000010FAC1711F4E0FC00E200930F0112D07C
:10096000BF91AF911F910F91FFBE189518951895E3
:10097000189518951895189518951895189518950F
:1009800018951895B1E0A0E000E000680ED010E1E5
:100990000D910ED01A95E1F700E4006806D010E141
:1009A0000D9106D01A95E1F70895459804D0089561
:1009B000459A01D00895299A0000000000000BB963
:1009C000000000000000299801E09ED008958F9358
:1009D0009F93AF93BF93CF9388279927AA27BB27CD
:1009E000C0E2000F111F221F331F881F991FAA1F6B
:1009F000BB1F84179507A607B70728F00395841B2C
:100A0000950BA60BB70BCA9561F7CF91BF91AF912C
:100A10009F918F9108950F931F932F933F93021BE4
:100A2000130B3F912F911F910F9108951F9310E386
:100A3000010F1F9108953F934F9340E0203021F024
:100A400034E6430F2A95E1F7103021F03AE0430FE6
:100A50001A95E1F7400F042F4F913F9108953F936E
:100A600034E620E02395031BE8F72A95030F3AE0CC
:100A700010E01395031BE8F71A95030F30E3230FDB
:100A8000130F030F3F9108952F93102F0F7012959E
:100A90001F7027E30A3008F420E3020F27E31A301F
:100AA00008F420E3120F2F9108954F935F936F93F3
:100AB0004427552760E1000F111F441F551F42179F
:100AC000530718F00395421B530B6A95A1F75F93E8
:100AD0004F932F913F916F915F914F9108951F9385
:100AE000F999FECF10E01FBB52BD41BD00BD653A74
:100AF00011F4FA9AF99A1F910895F999FECF52BD0F
:100B000041BDF89A00B508951F932F93A8952BE146
:100B100019E11A95F1F72A95D9F70A95B9F72F91A6
:040B20001F91089584
:00000001FF
